:100000000C945B000C9483000C9483000C9483008C
:100010000C9483000C9483000C9483000C94830054
:100020000C9483000C9483000C9483000C94830044
:100030000C9483000C9483000C9483000C94830034
:100040000C9478010C9483000C945D030C94830051
:100050000C9483000C9483000C9483000C94830014
:100060000C9483000C948300000024272A000025B0
:10007000282B000023262904040404040404040299
:100080000202020202030303030303010204081035
:100090002040800102040810200102040810200002
:1000A0000000070002010000030406000000000039
:1000B00000000000770111241FBECFEFD4E0DEBFA7
:1000C000CDBF11E0A0E0B1E0E2ECF9E002C00590A4
:1000D0000D92A230B107D9F711E0A2E0B1E001C062
:1000E0001D92AB38B107E1F710E0C6EBD0E004C0D9
:1000F0002297FE010E94DC04C43BD107C9F70E948D
:10010000AB000C94E0040C9400000F931F938091BB
:1001100000010E944C0202E011E0BC01C8010E94F3
:100120004501C8010E94CE0062E370E080E090E0EB
:100130000E94B5011F910F91089560E08091000128
:100140000E942E0240E855E260E070E082E091E01B
:100150000E94710108950E94E4010E949D000E9486
:100160008500FDCF08950895CB01BA0133274427B8
:1001700055270E94A30308952AE00E94B400089521
:10018000AB01662777270E94BC000895862F0E9446
:100190009B030895862F0E949B0308950F931F933E
:1001A0008C016DE00E94CA006AE0C8010E94CA008A
:1001B0001F910F9108950F931F938C010E94BC0013
:1001C000C8010E94CE001F910F9108950F931F93B5
:1001D0008C010E94C600C8010E94CE001F910F91A1
:1001E00008950F931F938C010E94CA00C8010E94BA
:1001F000CE001F910F910895EF92FF920F931F93DE
:10020000CF93DF93EC017A018B0177FF0BC06DE296
:100210000E94CA0010950095F094E094E11CF11C36
:10022000011D111D2AE0B801A701CE010E94B400F2
:10023000DF91CF911F910F91FF90EF9008950F9351
:100240001F938C010E94FC00C8010E94CE001F91E8
:100250000F9108952115310521F4642F0E94CA00E1
:1002600008952A30310519F40E94FC0008950E9477
:10027000B40008950F931F938C010E942A01C801B6
:100280000E94CE001F910F910895AB01662757FD84
:100290006095762F0E94FC0008950F931F938C01A8
:1002A0000E944501C8010E94CE001F910F91089540
:1002B000CB010E94690408950F931F938C010E9443
:1002C0005801C8010E94CE001F910F9108950E940D
:1002D000540308950E94350308950E94240399272A
:1002E0000895CB01BA010E94E3020895089508958C
:1002F0001F920F920FB60F9211248F939F93AF937B
:10030000BF938091070190910801A0910901B091DC
:100310000A010196A11DB11D809307019093080168
:10032000A0930901B0930A01BF91AF919F918F9162
:100330000F900FBE0F901F9018956091070170915C
:1003400008018091090190910A0127E0660F771F4B
:10035000881F991F2A95D1F72DE730E040E050E043
:100360000E948904CA01B9010895AF92BF92CF9249
:10037000DF92EF92FF920F931F935B016C010E943B
:100380009D017B018C010E949D016E197F09800BEC
:10039000910B6A157B058C059D05A8F31F910F91A4
:1003A000FF90EF90DF90CF90BF90AF9008950197AE
:1003B00051F0880F991F880F991F02972FB7F89453
:1003C0000197F1F72FBF08957894109207011092CA
:1003D00008011092090110920A0184B5826084BD5F
:1003E00084B5816084BD85B5826085BD85B5816039
:1003F00085BDEEE6F0E0808181608083E1E8F0E099
:10040000808182608083808181608083E0E8F0E089
:10041000808181608083E1EBF0E080818460808373
:10042000E0EBF0E0808181608083ECE7F0E08081A8
:100430008F778083808180648083EAE7F0E0808129
:1004400084608083808182608083808181608083FA
:100450008081806880831092C1000895282F3327FF
:10046000C90185579F4FFC01949129583F4FF901CD
:100470008491882381F0E82FFF27E859FF4FE4910A
:10048000FF27662329F4808190958923808308952E
:100490008081892B80830895482F5527CA01815672
:1004A0009F4FFC012491CA0185579F4FFC019491F5
:1004B00049585F4FFA013491332319F480E090E0FA
:1004C0000895222331F1233021F4809180008F7729
:1004D00005C0243031F4809180008F7D80938000AE
:1004E00018C0213019F484B58F7704C0223021F46C
:1004F00084B58F7D84BD0DC0263021F48091B0007D
:100500008F7705C0273029F48091B0008F7D8093CC
:10051000B000E32FFF27EE58FF4FE491FF278081C3
:1005200020E030E0892311F021E030E0C901089596
:10053000482F5527CA0181569F4FFC012491CA01BB
:1005400085579F4FFC01949149585F4FFA013491B0
:100550003323C1F1222331F1233021F48091800033
:100560008F7705C0243031F4809180008F7D809397
:10057000800018C0213019F484B58F7704C0223070
:1005800021F484B58F7D84BD0DC0263021F4809187
:10059000B0008F7705C0273029F48091B0008F7D9F
:1005A0008093B000E32FFF27E359FF4FE491FF272B
:1005B000662329F480819095892380830895808122
:1005C000892B80830895EF92FF920F931F937B01F5
:1005D0008C0122E030E040E050E00E94AB04205C5F
:1005E0003D4B404F5F4FCA01B901A80197010E94DE
:1005F000AB042150304040405040BB2757FDBA95D6
:10060000A52F942F832F2F5F3F4F4F4F5F4F809326
:10061000C50021502093C400E1ECF0E080818061AE
:1006200080838081886080838081806880831F913F
:100630000F91FF90EF900895982F8091C00085FF53
:10064000FCCF9093C600089580910301909104011E
:100650002091050130910601821B930B80589F4F1A
:1006600060E870E00E947604089540910501509181
:10067000060180910301909104018417950719F4F4
:100680008FEF9FEF0895FA01E55FFE4F2081CA01C9
:10069000019660E870E00E947604909306018093D2
:1006A0000501822F992708958091050190910601F7
:1006B000909304018093030108951F920F920FB647
:1006C0000F9211242F933F934F935F936F937F93D8
:1006D0008F939F93AF93BF93EF93FF934091C60087
:1006E000E0910301F0910401CF01019660E870E010
:1006F0000E9476049C0180910501909106012817C3
:10070000390739F0E55FFE4F4083309304012093B1
:100710000301FF91EF91BF91AF919F918F917F91D5
:100720006F915F914F913F912F910F900FBE0F905E
:100730001F9018950895982F8091C00085FFFCCFD9
:100740009093C60008952F923F924F925F926F92BE
:100750007F928F929F92AF92BF92CF92DF92EF9251
:10076000FF920F931F93CF93DF93CDB7DEB7A09780
:100770000FB6F894DEBF0FBECDBF6B017C0129011F
:100780003A01611571058105910541F48091C00020
:1007900085FFFCCF80E38093C60041C08824992464
:1007A00054011E010894211C311C8101080D191DE2
:1007B000C701B601A30192010E948904F801608378
:1007C0000894811C911CA11CB11CC701B601A30196
:1007D00092010E94890469017A01211531054105C0
:1007E000510519F79E012F5F3F4F14C008948108EF
:1007F0009108A108B108F901E80DF91DE081EA307E
:1008000010F4E05D01C0E95C8091C00085FFFCCF81
:10081000E093C60081149104A104B10439F7A096B5
:100820000FB6F894DEBF0FBECDBFDF91CF911F9101
:100830000F91FF90EF90DF90CF90BF90AF909F907F
:100840008F907F906F905F904F903F902F90089582
:1008500020E130E040E050E00E94A303089528E04A
:1008600030E040E050E00E94A303089522E030E031
:1008700040E050E00E94A30308958091C00085FFEE
:10088000FCCF8AE08093C6000895EF92FF920F9309
:100890001F937B018C0197FF0FC08091C00085FFE3
:1008A000FCCF8DE28093C60010950095F094E09403
:1008B000E11CF11C011D111D2AE030E040E050E078
:1008C000C801B7010E94A3031F910F91FF90EF9001
:1008D0000895FC0107C08091C00085FFFCCF3196D0
:1008E0009093C60090819923B1F7089597FB092E44
:1008F00007260AD077FD04D049D006D000201AF48C
:10090000709561957F4F0895F6F7909581959F4F6B
:100910000895A1E21A2EAA1BBB1BFD010DC0AA1F40
:10092000BB1FEE1FFF1FA217B307E407F50720F058
:10093000A21BB30BE40BF50B661F771F881F991FD3
:100940001A9469F760957095809590959B01AC011C
:10095000BD01CF01089597FB092E05260ED057FD46
:1009600004D0D7DF0AD0001C38F45095409530955C
:1009700021953F4F4F4F5F4F0895F6F79095809523
:10098000709561957F4F8F4F9F4F0895AA1BBB1B9A
:1009900051E107C0AA1FBB1FA617B70710F0A61B7F
:1009A000B70B881F991F5A95A9F780959095BC01A0
:1009B000CD010895EE0FFF1F0590F491E02D0994ED
:0209C000FFCF67
:0209C2000C0027
:00000001FF
